:100000001E29A601A801A7000130A4002808260285
:10001000031D0C282708250204300318013003199A
:1000200002302405031D01301A292016201E20123B
:10003000A01A1E28A01654200318492820110830A1
:10004000A8006520A70DA80B212820192E28201A0A
:100050002A287A2074207020201A49207720031043
:10006000270850282016201E2012201B3C28FE396D
:10007000A400201703105028A01B4428AD00A0178F
:100080005420031849282D08582003184928201EF9
:1000900050287A2074202013A013A012201177205A
:1000A0002F14031C2F101A296D202408A01A0138C0
:1000B000A7000830A800A70D7720031860287A2031
:1000C00074207020A80B5B287720742067286400B8
:1000D00003108619031470200800772074207A20FA
:1000E0000611831606117D28831606157D288316B2
:1000F00086157D28861183168611831208008317C2
:100100008001840AFF3E031D80281A29A801A70048
:10011000FF30A707031CA807031C1A290330A600F9
:10012000DF3094208828A601E83EA500A609FC300F
:10013000031C9D28A50703189A28A5070000A60FF1
:100140009A282518A328A51CA7280000A72808007E
:100150008316861483128313AE01AD012930840007
:100160000130A600B8309420861816290330A60066
:1001700072309420AE0A21302E020318C9280314CD
:1001800086180310800DAD0AAD1DB628840AAD0196
:10019000B62829308400A201AD01A601A501800D79
:1001A000A20D800DA20DAD0A0B2124191629A40C55
:1001B000A201800DA20D800DA20DAD0A0B21241904
:1001C0001629A40C0530A300A201800DA20D800DFC
:1001D000A20DAD0A2D1DEE28840AAD010B212419B4
:1001E0001629A40CA60DA30BE4280630A300A20137
:1001F000800DA20D800DA20DAD0A2D1D0129840ACE
:10020000AD010B2124191629A40CA50DA30BF72869
:10021000250803101A29A401220B10292414080010
:10022000023022020319080024150800FF30A6003E
:10023000A50003148313831203130800A0010730E1
:100240009F0083168501C230860020308400603014
:1002500083128020A0308400503080202030840021
:1002600030307F20D0303420003034201520B400CE
:10027000B41F4129B413D030342000303420340866
:1002800032207C2BB508031D4C293608B300061418
:100290000511851106126E2901303502031D5729FB
:1002A0003708B30005150610061285116E290230B5
:1002B0003502031D62293808B300851506120511A1
:1002C00006106E2903303502031D6D293908B3006D
:1002D00006168511051106106E29B5018310331815
:1002E000831483180517831C05138310B318831414
:1002F00083180514831C0510831033198314831885
:100300008514831C85108310B319831483188517F3
:10031000831C851308000614051585150616033081
:10032000A800E83087200614B5014221A820B100BA
:100330002608B200310A03199629B108031DA22923
:10034000B601AF2901303102031DA9290130B600E1
:10035000AF2902303102031DAF290230B60005304B
:1003600032020130031D0030B0000B303102013089
:10037000031D0030B0050319C32906100330A8007F
:10038000E8308720C429932905150130B5000230D3
:1003900036020130031D0030B0003708A5000330DD
:1003A0000120B0050319D529B70142210330A80067
:1003B00020308720A820B1002608B200310A031996
:1003C000DA2902303602031DFF29B108031DEA298C
:1003D000B701FE2901303102031DF1290130B700B8
:1003E000FE2902303102031DF8290230B700FE2930
:1003F00003303102031DFE290330B700422AB10841
:10040000031D042AB701422A01303102031D0B2AC1
:100410000130B700422A02303102031D122A023095
:10042000B700422A03303102031D192A0330B700F6
:10043000422A04303102031D202A0430B700422A28
:1004400005303102031D272A0530B700422A063045
:100450003102031D2E2A0630B700422A073031022E
:10046000031D352A0730B700422A08303102031D28
:100470003C2A0830B700422A09303102031D422AC3
:100480000930B700053032020130031D0030B000E2
:100490000B3031020130031D0030B0050319562A1C
:1004A00005110330A800E8308720572AC429851594
:1004B0000230B50042210330A80020308720A82058
:1004C000B1002608B200310A03195F2AB108031DE2
:1004D0006B2AB8018D2A01303102031D722A0130C6
:1004E000B8008D2A02303102031D792A0230B8008B
:1004F0008D2A03303102031D802A0330B8008D2A73
:1005000004303102031D872A0430B8008D2A0530DB
:100510003102031D8D2A0530B8000530320201304A
:10052000031D0030B0000B3031020130031D0030DC
:10053000B0050319A12A85110330A800E8308720EF
:10054000A22A572A06160330B50042210330A8001C
:1005500020308720A820B1002608B200310A0319F4
:10056000AA2AB108031DB62AB901F42A01303102C2
:10057000031DBD2A0130B900F42A02303102031DE7
:10058000C42A0230B900F42A03303102031DCB2AF9
:100590000330B900F42A04303102031DD22A04309A
:1005A000B900F42A05303102031DD92A0530B900FB
:1005B000F42A06303102031DE02A0630B900F42A7D
:1005C00007303102031DE72A0730B900F42A08304A
:1005D0003102031DEE2A0830B900F42A0930310235
:1005E000031DF42A0930B900053032020130031D21
:1005F0000030B0000B3031020130031D0030B00577
:100600000319082B06120330A80020308720092B7D
:10061000A22A061485150130A800F43087203A1765
:10062000381D3A13BA16B81CBA123A16381C3A12C8
:10063000BA15B91DBA113A15391D3A11BA14B91CB7
:10064000BA103A14391C3A103B13BB16B61CBB1235
:100650003B16361C3B12BB15B71DBB113B15371D96
:100660003B11BB14B71CBB103B14371C3B10D030E4
:100670003420013034203A0832200F308620D03028
:100680003420023034203B0832200F3086207C2B6F
:10069000D0303420013034201520BA00D03034203E
:1006A000023034201520BB0038153A1F3811B81419
:1006B000BA1EB81038143A1E3810B915BA1DB9113F
:1006C00039153A1D3911B914BA1CB91039143A1C2C
:1006D0003910B614BB1EB61036143B1E3610B715B3
:1006E000BB1DB71137153B1D3711B714BB1CB71015
:1006F00037143B1C3710080048234221BE01BD01BE
:100700000B303E02031C8A2B031DA12BB9303D0286
:100710000318A12BA820B1002608B2000530320230
:100720000130031D0030B000373031020130031DAD
:100730000030B00503199D2B8B29BD0A0319BE0F8C
:10074000802BB50A04303502031DA72BB5017C2B85
:02075000A82BD4
:02400E00703F01
:00000001FF
